:100000000C942A001895000018950000189500001F
:10001000189500001895000018950000189500002C
:10002000189500001895000018950000189500001C
:10003000189500001895000018950000189500000C
:1000400018950000189500001895000018950000FC
:10005000189500008FE58DBFC8E3E0E24E2E84E0E6
:100060008EBFD4E0F4E05F2EA89584B7082E877F7A
:1000700084BF88E1992781BD91BDEEEFF3E0A0E652
:10008000B0E088278D933197E9F787E689B980E05A
:1000900080BD88E18AB90E94ED01662487E886B9AF
:1000A00080E087B98FEF87BB379A8CE00E943B02D4
:1000B0000E94D8018FE711E00E94E701EEEFF5E022
:1000C0000E94D1018FEB11E00E94E701EEEFF5E015
:1000D0000E94D10183E911E00E94E701EEEFF5E013
:1000E0000E94D10183ED11E00E94E701EEEFF5E0FF
:1000F0000E94D101E4E1F6E00E94C3010E94CA011E
:100100000E94B701A2E6B0E08D9388278C93A2E607
:10011000B0E00E94BD010E94CA01A2E6B0E0ECE29C
:10012000F6E00E94EB0211F00C94FC0080E090E0FD
:10013000A0E6B0E08D939C93A0E6B0E00D911C91F9
:10014000073050E015071CF011F00C94C30007B104
:10015000007E8091600090E0890F082707B90E9417
:100160007702A0E6B0E0AD90BD90A4E6B0E0AA0CA6
:10017000BB1CAA0DBB1D8D939C93A0E6B0E00E9412
:10018000B0010C949C00EEE2F6E00E94C3010E94D4
:10019000CA0180E090E0A0E6B0E08D939C93A0E6D9
:1001A000B0E00D911C91073050E015071CF011F0E4
:1001B0000C94F600A8E0B4E0E0E6F0E0A190B19085
:1001C000E4E6F0E0AA0CBB1CEA0DFB1D0E949202C3
:1001D0000E94BB01E0E3F6E00E94C3010E94CA0155
:1001E000A0E6B0E00E94B0010C94CF00E2E3F6E09C
:1001F0000E94C3010E94CA01A2E6B0E0E4E3F6E077
:100200000E94EB0211F00C940801C09A0C941201A8
:10021000A2E6B0E0E6E3F6E00E94EB0211F00C94F7
:100220001201C098A2E6B0E0E8E3F6E00E94EB021B
:1002300011F00C941E01C19A0C942801A2E6B0E0C2
:10024000EAE3F6E00E94EB0211F00C942801C19859
:10025000A2E6B0E0ECE3F6E00E94EB0211F00C94B1
:100260003401C29A0C943E01A2E6B0E0EEE3F6E05F
:100270000E94EB0211F00C943E01C298A2E6B0E09D
:10028000E0E4F6E00E94EB0211F00C944A01C39AFC
:100290000C945401A2E6B0E0E2E4F6E00E94EB0226
:1002A00011F00C945401C398A2E6B0E0E4E4F6E047
:1002B0000E94EB0211F00C946001C49A0C946A0144
:1002C000A2E6B0E0E6E4F6E00E94EB0211F00C9446
:1002D0006A01C498A2E6B0E0E8E4F6E00E94EB020E
:1002E00011F00C947601C59A0C948001A2E6B0E05E
:1002F000EAE4F6E00E94EB0211F00C948001C5984C
:10030000A2E6B0E0ECE4F6E00E94EB0211F00C94FF
:100310008C01C69A0C949601A2E6B0E0EEE4F6E0F9
:100320000E94EB0211F00C949601C698A2E6B0E090
:10033000E0E5F6E00E94EB0211F00C94A201C79AEE
:100340000C94AC01A2E6B0E0E2E5F6E00E94EB021C
:1003500011F00C94AC01C7980C948000F894FFCF76
:10036000ED91FC91EF5FFF4FFC93EE9308955F9B3F
:10037000FECF8CB10895A8E0B4E08D91882311F0F0
:100380000CD0FBCF08950E948002802D11F005D083
:10039000FACF08958DE001D08AE05D9BFECF8CB945
:1003A00008950E948002802D11F05FD0FACF089549
:1003B00081E061D00FD080E85EC08FE7213039F056
:1003C0008FEB223021F083E9233009F083ED810F98
:1003D0000C943B0283E099277BC08AEF90E00E9457
:1003E0006802A79AA69AA59AA49AA29AA19AA998ED
:1003F00085E090E00E946802AA98AF98AE98AD9A06
:10040000AC9AAA9AEF93FF93ECE8F1E00E945C02A9
:10041000FF91EF91AA9859D0AA9AEF93FF93ECE835
:10042000F1E00E945C02FF91EF91AA984ED0AA9A47
:10043000EF93FF93ECE8F1E00E945C02FF91EF91F3
:10044000AA9843D0AC98AA9AEF93FF93ECE8F1E016
:100450000E945C02FF91EF91AA9837D088E20BD0FE
:100460008EE009D086E007D00895A99A829505D03C
:1004700004D02BD00895A998F9CF859510F4AC9AA3
:1004800001C0AC98859510F4AD9A01C0AD988595E2
:1004900010F4AE9A01C0AE98859510F4AF9A01C0E1
:1004A000AF98AA9AEF93FF93ECE8F1E00E945C0208
:1004B000FF91EF91AA9808953197F1F70895689404
:1004C00062F80895E89462F8089581E090E000C031
:1004D000EF93FF93EE27E82BE92B31F0E0EAFFE002
:1004E0003197F1F70197D1F7FF91EF910895369A7F
:1004F0003699FECF369A3699FECF84B195B10895DC
:10050000C895319600200895000F111F221F331F38
:10051000089500951095209530950F5F1F4F2F4F30
:100520003F4F0895019110810EC0019111912191C9
:1005300030810BC00191108117FF05C03FEF2FEFF5
:1005400004C0008111272227332737FF03C0E1DFD2
:100550008DE28D93CF93DF93CF92DF92EF92AA2417
:10056000BB24CC24DD24EE2440E2CAE0DD2755E0A4
:1005700093E38881890F87FD9F7083FD907F891B9E
:1005800089935A95A9F7C0DFAA1CBB1CCC1CDD1CA3
:10059000EE1C4A9551F7E894EFE0FF2782910ED0C8
:1005A000EB30E0F71EF068948A2D0CD088278D93ED
:1005B000EF90DF90CF90DF91CF910895982F8295A3
:1005C00001D0892F8F70805D26F0803309F4089563
:1005D00068948D930895689401C0E894AF93BF9395
:1005E0008D9116F0919103C00E948002902D891781
:1005F00018F011F48823A1F7BF91AF9108954141FC
:1006000041414141414141414141414141414141DA
:100610004141000048454C4C4F205445524D494EF5
:10062000414C2121212121212121000071005B0069
:100630003A005D0041006100530073004400640013
:100640004600660047006700480068004A006A00EC
:040650004B006B00F0
:00000001FF
